:1000000000308A006F2900000A108A100A11820746
:1000100028340C34013406340A108A100A1182077D
:10002000413454342B3443344D3447344C343D3410
:1000300031340D3400343130840083130008031947
:1000400032280130F800BF30F7006400F70B252894
:10005000F80B23284A30F700F70B2C280000640027
:10006000800B212800340708F039B80037080F3911
:100070003804870006148316061064002030F70049
:10008000F70B4028432883120610831606108312AC
:100090000034B508031D4E2886104F288614831699
:1000A00086108312B60E3608B7003320B60E360817
:1000B000B700332064004230F700F70B5D280034AE
:1000C0001430B1001B20F030831687058312861090
:1000D0008316861083120610831606108312AA0157
:1000E0002A08023C031C7C280230B1001B2003308C
:1000F000B7003320AA0A702864000C30F700F70B11
:100100007F2882280230B700332064000C30F700CB
:10011000F70B88288B28AA012A08023C031C9C287C
:100120002A080420AB00B5012B08B6004920023094
:10013000B1001B20AA0A8C28C02901303202FC3EE3
:100140000318AF28043EBA28B301AF284030B300EB
:10015000AF281430B300AF285430B300AF280130BB
:100160003102B30733088038B400B5013408B60053
:10017000492000340A108A100A118207A428A628F0
:10018000A928AC2830080C3A0319D028063A0319DC
:10019000D828073A0319DE28053A0319E328E82886
:1001A000B5010130B60049200230B1001B20F4280F
:1001B0000130B1000230B2009D20F4280130B100BE
:1001C000B2009D20F428B5011030B6004920F42873
:1001D00030081F3C031CEE280730B0050130B50085
:1001E0003008B6004920F42800343108F801300204
:1001F0000318FD283008F7000929F7010830B2007C
:10020000B00DF70D310877020318F700F80DB20BA7
:100210000029003420302B1E3030AC002A08F700B3
:10022000AA1F1929F709F70A7708AA002D30AC0090
:10023000AB172A08B0006430B100F5207708AA0097
:1002400030307807AD002A08B0000A30B100F52040
:1002500030307707AF0030307807AE002C08F70059
:10026000AB1D3429AB1F2B112B1A4129AB1F5C2965
:100270002B195C297708AD00AB185C297708AE0014
:100280005C2930302D02031D5C297708AD00203039
:10029000AC00AB1D4F292B11AB14AB1FAB10303092
:1002A0002E02031D5C297708AE002030AD00AB1D87
:1002B0004F29AB10AB1F2B102B1D61292C08B00050
:1002C000C220AB1C66292D08B000C2202B1C6B2954
:1002D0002E08B000C2202F08B000C220292A8401B5
:1002E00083131F3083050C3083169900A6309800C5
:1002F00090308312980083161F149F141F159F11AE
:1003000007309C00FF308312A00083161F149F1437
:100310001F159F1183121F10831609128312941246
:10032000A012200883168700831220162008831647
:1003300087008312A01120088316870001308312E2
:1003400094000030831694000108C73908388100F2
:10035000831290010030F800920000308316920062
:1003600007309C00050864000230F700F70BB6293F
:10037000B9291C0883120D1383169D01831260286E
:100380006430B1001B20AA012A080C20AA0AF70039
:1003900077080C1EC92999000A302A02031DC429B6
:1003A0002130840083138403840A8C1ED5291A0803
:1003B00080000D300002031DD42980018C1EDE292F
:1003C0001A088C1EE1291A08213084008313840343
:1003D000840A8C1EE9291A0880000D300002031DD2
:1003E000E8298001A9012908363C031CFC298C1E40
:1003F000F7291A08A90AF3292130840083138403FA
:10040000840A8C1E012A1A0880000D300002031D88
:10041000002A800121308400831300300004031976
:10042000212AAB010408AA002B10831B2B140008FF
:10043000B000C2202A08840083132B188317840A73
:100440000D2A0A30B000C2202108AA001F30AB00DC
:040450000A29630012
:02400E00393F38
:00000001FF
